:020000020000FC
:0200000049C0F5
:020016003CC0EC
:10001A0000C04F935F935FB74091670045300CF47F
:10002A0003C0442740936700403041F49398949862
:10003A009598929A009166007ED05DD0413041F445
:10004A00929894989598939A0091650074D053D099
:10005A00423041F4929893989598949A009164004A
:10006A006AD049D0433041F4929893989498959ADB
:10007A000091630060D03FD04395409367005FBF13
:10008A005F914F911895019618950FED0DBF0CE7EA
:10009A0001BB01EC07BB0CE108BB00E20BBF0CE1A2
:1000AA0000BD02E000BF05E003BF09E106BF01E0B1
:1000BA0009BF11241092670080E090E0789425D05F
:1000CA004FD040D03FD03ED03DD03CD03BD0F7CFF0
:1000DA00EE24FF1841E1001F111F4A9509F4089503
:1000EA00EE1CFF1CE21AF30A20F4E20EF31E8894B7
:1000FA00F2CF0894F0CF0FB800E40EB90BE10DB9B6
:10010A00769BFDCFC09AC098089554E0A3E6B0E06C
:10011A0080936100909362000091610010916200E7
:10012A002AE030E0D5DFED9200936100109362007F
:10013A005A9591F70895ECE7F1E01127E00FF11FC6
:10014A00049008950F931F930FEF1FEF1A95000065
:10015A0000000000D9F70A95C1F71F910F91089581
:10016A000F931F9300E412B3102712BB1F910F9134
:0E017A000895C0F9A4B0999282F880909C007C
:00000001FF
